:100000000C948A070C94A7070C94A7070C94A707D5
:100010000C94A7070C94A7070C94A7070C94A707A8
:100020000C94A7070C94A7070C94A7070C94A70798
:100030000C94A7070C94A7070C94A7070C94B70778
:100040000C94A7070C94A7070C94780C0C94A707A2
:100050000C94A7070C94A7070C94A7070C94A70768
:100060000C94A7070C94A7070C94A7070C94A70758
:100070000C94A7070C94A7070C94A7070C94A70748
:100080000C94A7070C94A7070C94A7070A0A0A5711
:10009000454C434F4D4520544F2054484520424441
:1000A0004D4943524F204D415652494320535045EC
:1000B000414B4A455420544553542050524F4752C7
:1000C000414D0A003E3E3E2000494E56414C4944B7
:1000D0000A00082008000A436F6D6D616E64733A70
:1000E0000A0A20203F20202020202020202020201D
:1000F000202020202020202D20746869732068652E
:100100006C70206D6573736167650A2020616E6E87
:100110006F756E6365202020202020202020202065
:100120002D20706C617920616E6E6F756E63652035
:100130006D6573736167650A20206C697374202094
:10014000202020202020202020202020202D206C56
:100150006973742070686F6E656D65206D6E65756E
:100160006D6F6E69637320616E6420636F64657385
:100170000A20206C69737476202020202020202003
:100180002020202020202D206C6973742070686F3F
:100190006E656D65206D6E65756D6F6E6963732C30
:1001A00020636F64657320616E642064657363729D
:1001B000697074696F6E730A20202020202020202F
:1001C000202020202020202020202020202020202F
:1001D0002028766572626F7365206C697374696E2E
:1001E00067290A2020736370203C61736369692D5D
:1001F000746578743E2020202D2069737375652006
:1002000053435020636F6E74726F6C206D6573730F
:100210006167657320746F20746865205370656131
:100220006B4A65740A2020776964203C73637265A9
:10023000656E2D77696474683E202D207365742087
:100240007468652073637265656E2077696474688D
:100250003B20757365642062792074686520276C83
:100260006973742720616E6420276C697374762724
:100270000A20202020202020202020202020202094
:100280002020202020202020202020636F6D6D6101
:100290006E647320746F2064657465726D696E6539
:1002A00020686F77206D75636820696E666F726D68
:1002B0006174696F6E2063616E0A20202020202007
:1002C000202020202020202020202020202020202E
:1002D00020202020666974206F6E206F6E65206C70
:1002E000696E652E0A20203C70686F6E656D657CB6
:1002F000636F64653E202E2E2E202D20706C617958
:10030000207468652073706563696669656420732D
:10031000657175656E63650A0A0091839104C388EF
:100320008C05C0A205A98605AA8000AE80008C9B22
:10033000C29489058C9AA69481C205BBC680C2046A
:10034000A583BF05BF83BBBF05C79489B394848CC5
:100350000070300070310070320070330070340073
:10036000703500703600697900696800657900654C
:1003700068006179006178007578006F68006177C6
:10038000006F77007568007577006D6D006E650011
:100390006E6F006E6765006E676F006C65006C6F56
:1003A00000777700727200697972720065797272F3
:1003B00000617872720061777272006F77727200FA
:1003C00065796979006F686979006F776979006F7D
:1003D00068696800697965680065686C6C006979AE
:1003E000757700617875770069687777006179774C
:1003F00077006F777777006A68007676007A7A0000
:100400007A6800646800626500626F006562006F70
:100410006200646500646F006564006F6400676576
:1004200000676F006567006F6700636800686500BC
:10043000686F00776800666600736500736F00730D
:1004400068007468007474007475007473006B65E0
:10045000006B6F00656B006F6B00706500706F0064
:1004600072300072310072320072330072340072E6
:100470003500723600723700723800723900613010
:100480000061310061320061330061340061350088
:100490006136006137006138006139006230006206
:1004A000310062320062330062340062350062362D
:1004B0000062370062380062390063300063310047
:1004C00063320063330063340063350063360063D6
:1004D00037006338006339006430006431006432EF
:1004E000006433006434006435006436006437000F
:1004F00064380064390064313000643131006D309B
:10050000006D31006D32006E7300666173740073AC
:100510006C6F77007374726573730072656C6178C9
:10052000007761697400736F667400766F6C756D27
:100530006500737065656400706974636800626566
:100540006E64007265706561740064656C61790049
:10055000726573657400306D732073696C656E63CA
:1005600065003130306D732073696C656E636500B2
:100570003230306D732073696C656E63650037309F
:10058000306D732073696C656E63650031306D7317
:100590002073696C656E6365202F77207472616EBD
:1005A000730033306D732073696C656E6365202F43
:1005B00077207472616E730036306D732073696CCE
:1005C000656E6365202F77207472616E73007365AA
:1005D000652C206576656E2C206665656400736900
:1005E000742C206669782C2070696E0068616972CD
:1005F0002C20676174652C206265696765006D65F4
:10060000742C20636865636B2C20726564006861DC
:10061000742C20666173742C2066616E00636F74A5
:1006200074656E006C75636B2C2075702C20756E74
:10063000636C6500686F742C20636C6F636B2C2097
:10064000666F78006661746865722C2066616C6CF8
:1006500000636F6D622C206F7665722C20686F6C62
:100660006400626F6F6B2C20636F756C642C207359
:10067000686F756C6400666F6F642C206A756E65B8
:10068000006D696C6B2C2066616D6F7573006E690F
:10069000702C2064616E6765722C207468696E002E
:1006A0006E6F2C20736E6F772C206F6E00746869EC
:1006B0006E6B2C2070696E670068756E672C2073F6
:1006C0006F6E67006C616B652C20616C61726D2CC4
:1006D000206C6170656C00636C6F636B2C20706CB8
:1006E00075732C2068656C6C6F00776F6F6C2C20B5
:1006F0007377656174007261792C20627261696E32
:100700002C206F76657200636C6561722C206865C1
:1007100061722C207965617200686169722C2073A6
:10072000746169722C207265706169720066697209
:100730002C20626972642C206275726E0070617286
:10074000742C206661726D2C207961726E00636F6B
:10075000726E2C20666F75722C20796F757200672F
:100760006174652C206174652C20726179006D695B
:1007700063652C2066696768742C207768697465E6
:1007800000626F792C20746F792C20766F69636515
:1007900000736B692C20666976652C2049007965A9
:1007A000732C207961726E2C206D696C6C696F6E90
:1007B00000736164646C652C20616E676C652C202D
:1007C0007370656C6C00637574652C2066657700CA
:1007D00062726F776E2C20636C6F776E2C2074685A
:1007E0006F7573616E640074776F2C206E65772C63
:1007F000207A6F6F006F75722C206F7563682C20E4
:100800006F776C00676F2C2068656C6C6F2C2073A1
:100810006E6F7700646F6467652C206A65742C20A6
:1008200073617661676500766573742C2065766503
:100830006E007A6F6F2C207A617000617A75726534
:100840002C207472656173757265007468657265D9
:100850002C20746861742C2074686973006265616F
:10086000722C20626972642C206265656400626F7C
:100870006E652C20626F6F6B2C2062726F776E003A
:100880006361622C20637269622C2077656200626A
:100890006F622C207375622C20747562006465652C
:1008A000702C20646174652C20646976696465002D
:1008B000646F2C20647573742C20646F6700636F01
:1008C000756C642C2062697264006275642C206609
:1008D0006F6F64006765742C20676174652C2067F6
:1008E0007565737400676F742C20676C75652C20B8
:1008F000676F6F007065672C2077696700646F67AA
:100900002C20706567006368757263682C206665CB
:1009100061747572652C206D617263680068656C26
:10092000702C2068616E642C206861697200686FA9
:10093000652C20686F742C206875670077686F2CB1
:10094000207768616C652C20776869746500666F34
:100950006F642C206566666F72742C206F6666006B
:100960007365652C20766573742C20706C7573002C
:10097000736F2C20737765617400736869702C2025
:1009800066696374696F6E2C206C656173680074AE
:1009900068696E2C206D6F6E746800706172742CC3
:1009A000206C6974746C652C2073697400746F2CEE
:1009B0002074616C6B2C2074656E007061727473AE
:1009C0002C20636F7374732C20726F626F747300CA
:1009D00063616E27742C20636C6F776E2C206B65BF
:1009E0007900636F6D622C20717569636B2C2066D2
:1009F0006F7800737065616B2C207461736B00629B
:100A00006F6F6B2C20746F6F6B2C206F63746F6231
:100A100065720070656F706C652C20636F6D70750A
:100A200074657200706F772C20636F707900726F3D
:100A3000626F7400726F626F7400726F626F740025
:100A4000726F626F7400726F626F7400726F626FA8
:100A50007400726F626F7400726F626F7400726FF5
:100A6000626F7400726F626F7400616C61726D000E
:100A7000616C61726D00616C61726D00616C6172BC
:100A80006D00616C61726D00616C61726D00616C12
:100A900061726D00616C61726D00616C61726D00FC
:100AA000616C61726D00626565707300626565708E
:100AB00073006265657073006265657073006265DE
:100AC00065707300626565707300626565707300C0
:100AD000626565707300626565707300626565705C
:100AE000730062696F6C6F676963616C0062696F44
:100AF0006C6F676963616C0062696F6C6F676963D3
:100B0000616C0062696F6C6F676963616C00626938
:100B10006F6C6F676963616C0062696F6C6F6769A6
:100B200063616C0062696F6C6F676963616C00621E
:100B3000696F6C6F676963616C0062696F6C6F6786
:100B40006963616C0062696F6C6F676963616C00F7
:100B500064746D660064746D660064746D66006430
:100B6000746D660064746D660064746D6600647410
:100B70006D660064746D660064746D660064746D07
:100B8000660064746D660064746D6600736F6E61F8
:100B9000722070696E6700706973746F6C2073687F
:100BA0006F7400776F77006E6F20736F756E6400DF
:100BB0002E352074696D6500312E352074696D65A0
:100BC0000073747265737320766F69636500726574
:100BD0006C617820766F6963650073746F70007262
:100BE000656475636520766F6C756D6520353020A2
:100BF00070637400302D3132372F393600302D318B
:100C000032372F31313400302D3235352F3838001E
:100C1000302D31352F3500302D32353500582A3101
:100C2000306D73007265736574207061726D73004E
:100C30000051035605015403620502570370050372
:100C40005A037E05045D038C05056003A205066357
:100C500003B805070A05B00B080F05B80B0E1405FD
:100C6000C10B0F1B05CE0B102105DA0B122605DF79
:100C70000B142B05F40B153205FD0B163805070C6C
:100C8000173E05100C1A4305170C1E4A051D0C1FB4
:100C90005005240C806603CE05816903DE05826C55
:100CA00003EC05836F03FE058472030E068575034E
:100CB0001D068678032406877B033406887E03445A
:100CC0000689810351068A840362068B87037606B0
:100CD0008C8A0381068D8D038E068E9003A0068F6D
:100CE0009303AD06909703B906919B03C406929EA9
:100CF00003D70693A103EA0694A403F60695A70377
:100D0000070796AC03190797B1032D0798B6033D63
:100D10000799BB034E079AC0035F079BC5036E0785
:100D20009CCA0381079DCF0391079ED4039E079F12
:100D3000D903B107A0DE03C607A1E303D007A2E8E9
:100D400003E707A3ED03F507A4F2030408A5F703DF
:100D50001408A6FA032708A7FD033208A800043BDD
:100D600008A903044B08AA06045D08AB09046E0831
:100D7000AC0C048008AD0F048F08AE12049D08AFC0
:100D80001504B008B01804BE08B11B04CA08B21E8E
:100D900004D408B32104E508B42404F408B52704F6
:100DA000FD08B62A040609B72D041D09B830042E23
:100DB00009B933043C09BA36044E09BB3904600949
:100DC000BC3C047009BD3F047A09BE42048F09BFD0
:100DD00045049B09C04804AD09C14B04BB09C24E80
:100DE00004D009C35104E209C45404F309C55704EB
:100DF000FF09C65A04130AC75D04240AC860042EFA
:100E00000AC96304340ACA66043A0ACB6904400A70
:100E1000CC6C04460ACD6F044C0ACE7204520ACF41
:100E20007504580AD078045E0AD17B04640AD27E25
:100E3000046A0AD38104700AD48404760AD587042C
:100E40007C0AD68A04820AD78D04880AD890048E38
:100E50000AD99304940ADA96049A0ADB9904A00A40
:100E6000DC9C04A60ADD9F04AC0ADEA204B20ADF01
:100E7000A504B80AE0A804BE0AE1AB04C40AE2AEC5
:100E800004CA0AE3B104D00AE4B404D60AE5B704FC
:100E9000DC0AE6BA04E20AE7BD04ED0AE8C004F899
:100EA0000AE9C304030BEAC6040E0BEBC904190BD1
:100EB000ECCC04240BEDCF042F0BEED2043A0BEF55
:100EC000D504450BF0D804500BF1DB04550BF2DED2
:100ED000045A0BF3E1045F0BF4E404640BF5E7043C
:100EE000690BF6EA046E0BF7ED04730BF8F0047867
:100EF0000BF9F3047D0BFAF604820BFBFA04870B63
:100F0000FCFE048C0BFD0105970BFE0405A30BFFF3
:100F10000705A70B11241FBECFEFD0E1DEBFCDBF69
:100F200011E0A0E0B1E0ECE2F9E200E00BBF02C0AA
:100F300007900D92A437B107D9F713E0A4E7B1E009
:100F400001C01D92AF32B107E1F70C94070C0C946D
:100F500000009C0112BE1092C9021092C80280913A
:100F6000C8029091C90282179307C9F708951F928A
:100F70000F920FB60F9211248F939F938091C80206
:100F80009091C90201969093C9028093C8029F91E3
:100F90008F910F900FBE0F901F90189513BE86B7BC
:100FA000836086BF87B7836087BF8DE083BF12BE33
:100FB00083E781BF08959C0144275527220F331FE3
:100FC000441F551F220F331F441F551F220F331F6D
:100FD000441F551F220F331F441F551F60E070E050
:100FE00081EE90E00E94281421503040832F9927F1
:100FF0008093900029B988E98AB908959C01442713
:101000005527220F331F441F551F220F331F441F24
:10101000551F220F331F441F551F220F331F441F1C
:10102000551F60E070E081EE90E00E94281421508E
:101030003040832F9927809398002093990088E06F
:1010400080939A000895882321F45D9BFECF6CB9AC
:101050000895813039F4EBE9F0E0808185FFFDCF20
:1010600060939C000895682F80E00E94230880E030
:1010700090E008950E9433080895682F81E00E944F
:10108000230880E090E008950E943D0808952F9283
:101090003F924F925F926F927F928F929F92AF9208
:1010A000BF92CF92DF92EF92FF920F931F93CF9355
:1010B000DF93682E882319F064E270E002C06BE0D1
:1010C00070E080916B0199270E9415145B0184E9FF
:1010D00090E00E9401141B0184E990E0B5010E9498
:1010E0000114892B19F00894211C311C12141304CB
:1010F0000CF09AC0442455248FC0C439D10508F09F
:1011000078C0CE01880F991F880F991F8C0F9D1FE3
:1011100020E33CE0FC01E20FF31F7490FC013196E8
:10112000E20FF31F459154910396820F931FFC0128
:10113000059114915F934F930F2EFAECCF2EF2E0AE
:10114000DF2EF02DDF92CF920E949C0F1F930F9302
:101150000AEA12E01F930F930E949C0F8DB79EB76F
:1011600008960FB6F8949EBF0FBE8DBF6620D9F0CB
:101170001F930F93DF92CF92872D99279F938F9381
:1011800080E091E09F938F9385EE92E09F938F9301
:101190000E946A0FEDB7FEB73A960FB6F894FEBFFD
:1011A0000FBEEDBF1AC08AEC92E09F938F93872DFC
:1011B00099279F938F9381E191E09F938F9385EE81
:1011C00092E09F938F930E946A0F8DB79EB7089607
:1011D0000FB6F8949EBF0FBE8DBF85EE92E09F9331
:1011E0008F930E94140F80E290E00E94630F0F9093
:1011F0000F900894E11CF11CC80DD91DAE14BF045A
:1012000009F07BCF8AE090E00E94630F0894411CB4
:10121000511C2414350441F01A141B049CF741019D
:10122000E201EE24FF2469CFDF91CF911F910F914E
:10123000FF90EF90DF90CF90BF90AF909F908F90F6
:101240007F906F905F904F903F902F900895CF9236
:10125000DF92EF92FF920F931F93CF93DF937C0166
:10126000C0E0D0E00F2EF0E3CF2EFCE0DF2EF02D1B
:10127000CE01880F991F880F991F8C010C0F1D1F1D
:10128000F8013196EC0DFD1D65917491C7010E9426
:10129000A00E892B39F4F801EC0DFD1DE4918E2F81
:1012A000992706C02196C439D10511F78FEF90E038
:1012B000DF91CF911F910F91FF90EF90DF90CF9032
:1012C0000895AF92BF92CF92DF92EF92FF920F9369
:1012D0001F93CF93DF93CDB7DEB722970FB6F89465
:1012E000DEBF0FBECDBF182F8D3019F08A3009F048
:1012F000F1C18AE00E94330866E971E0E09174016F
:10130000F0917501E60FF71F1082809196018823F6
:1013100009F4D3C1FB0105C031968081882309F40B
:10132000CCC18032C9F38C35B9F38C32A9F31AC21F
:101330000894E11CF11CD7011C91112331F01032EB
:1013400021F01C3511F01C3299F7EE16FF0609F456
:10135000B4C1D7011C92C0906C01D0906D01BF0147
:10136000C6010E94BD0E812FF7011083112341F4A5
:101370000EC00894E11CF11CD7018C91882339F030
:101380008032B9F38C35A9F38C3299F302C0EE2484
:10139000FF246AE171E0C6010E94B30E892B49F473
:1013A00086ED90E09F938F930E94340F0F900F90E3
:1013B00084C16CE171E0C6010E94B30E892BA9F5CE
:1013C00085E291E09F938F930E94140F8AE193E04E
:1013D0007C010F900F900F2EFFE2AF2EF1E0BF2E99
:1013E000F02D0F2EF7E3CF2EDD24F02DC80ED91EE1
:1013F000F7011491812F99279F938F93BF92AF92FA
:101400000E94140F612F81E00E9423080894E11CC0
:10141000F11C0F900F900F900F90CE14DF0441F746
:101420008AE090E00E94630F48C163E371E0C60167
:101430000E94B30E892B61F48AE090E00E94630F52
:1014400080E00E9447088AE090E00E94630F35C167
:1014500068E371E0C6010E94B30E892B61F48AE053
:1014600090E00E94630F81E00E9447088AE090E0CC
:101470000E94630F22C16EE371E0C6010E94B30EA9
:10148000892B91F580919601882389F4A1C1089454
:10149000E11CF11CD7018C91882379F4E114F1044B
:1014A00009F40BC1F7016081662371F406C10F2EA8
:1014B000F6E9EF2EF1E0FF2EF02D803241F38C356E
:1014C00031F38C3221F3EACF81E00E9423080894A3
:1014D000E11CF11CE114F10409F4EFC0D7016C9197
:1014E000662309F4EAC0F0CF62E471E0C6010E940D
:1014F000B30E892B09F045C0E114F10491F1F70115
:101500008081882341F40DC00894E11CF11CD701AF
:101510008C91882331F08032B9F38C35A9F38C3269
:1015200099F340E050E0BE016F5F7F4FC7010E941A
:10153000730D29813A812115310581F02E153F0562
:1015400069F4FF92EF9286E491E09F938F930E945B
:10155000140F0F900F900F900F90AFC060936B011E
:10156000ACC080916B0199279F938F938DE591E09B
:101570009F938F930E94140F0F900F900F900F90D6
:101580009CC085E291E09F938F930E94140F8091FD
:1015900096010F900F90882309F421C10F2EF6E9D0
:1015A000EF2EF1E0FF2EF02D07C00894E11CF11C96
:1015B000F7018081882331F08032B9F38C35A9F3AB
:1015C0008C3299F3E114F10409F473C0D7018C91C2
:1015D000882309F0DAC06DC00894C11CD11CF60143
:1015E0001081112341F0103231F01C3521F01C32F2
:1015F00099F701C06701B12ED6011C92FF92EF92BC
:1016000087E691E09F938F930E94140FF7018081EA
:10161000992787FD9095C0970F900F900F900F908E
:101620000A9788F440E050E0BE016F5F7F4FC7012A
:101630000E94730D062F89819A81009741F08E15C3
:101640009F0529F4B6C0C7010E942709082F802FE3
:1016500099279F938F938FE291E09F938F930E949E
:10166000140F0F900F900F900F900F3F21F0602FED
:1016700081E00E9423088B2DD601BC92112311F426
:1016800076010FC0760107C00894E11CF11CF70138
:101690008081882331F08032B9F38C35A9F38C3204
:1016A00099F3E114F10429F0D7018C91882309F012
:1016B0006CC08AE090E00E94630F84EC90E09F93FE
:1016C0008F930E94340F10927501109274010F9045
:1016D0000F908CC08830E1F4809174019091750175
:1016E000892B09F483C082ED90E09F938F930E9431
:1016F000340FE0917401F09175013197F093750109
:10170000E0937401EA56FE4F10820F900F906EC066
:101710000E9433088091740190917501FC01EA5692
:10172000FE4F108301969093750180937401805051
:10173000914009F05BC010927501109274011092F3
:10174000960189EC90E09F938F930E94340F84EC74
:1017500090E09F938F930E94340F0F900F900F9003
:101760000F9044C08081803209F4A7CF8C3509F4F2
:10177000A4CF8C3209F4A1CF7F010894E11CF11CA5
:101780001181112309F0DBCDE0CDF701108110327A
:1017900009F430CF1C3509F42DCF1C3209F42ACFBF
:1017A00067010894C11CD11C1181112309F01BCFC2
:1017B00022CF8FEF90E09F938F938FE291E09F93E2
:1017C0008F930E94140F0F900F900F900F9053CF94
:1017D0000F2EF6E9EF2EF1E0FF2EF02D63CE0F2E47
:1017E000F6E9EF2EF1E0FF2EF02DF0CE22960FB6A7
:1017F000F894DEBF0FBECDBFDF91CF911F910F9147
:10180000FF90EF90DF90CF90BF90AF900895CFEF13
:10181000D0E1DEBFCDBF0E94CE0740E250E066E7D8
:1018200071E08AED92E00E94CC0C80E895E20E9483
:10183000DB0780E895E20E94FE07789460E070E0A4
:101840008AE398E00E94C40E60E070E084E498E0CF
:101850000E94C40E90932203809321038AEF90E0AC
:101860000E94A9078CE890E09F938F930E94340F09
:101870008AE193E0EC010F900F908C01095C1F4FFF
:10188000FE01649181E00E9423082196C017D107D0
:10189000B9F786ED90E09F938F930E94340F84EC0C
:1018A00090E09F938F930E94340F0F900F900F90B2
:1018B0000F908091E40280FFFCCFF8948091E402C5
:1018C0008E7F8093E40278948091DC029091DD0217
:1018D000892B79F3CAEDD2E0CE010E94A60C0E94BA
:1018E00061098091DC029091DD02892B11F3F4CF24
:1018F0001F920F920FB60F9211242F933F934F9385
:101900005F936F937F938F939F93AF93BF93EF9367
:10191000FF936CB15C9909C08AED92E00E94E60CDD
:101920008091E40281608093E402FF91EF91BF9186
:10193000AF919F918F917F916F915F914F913F9167
:101940002F910F900FBE0F901F901895CF93DF939C
:10195000DC01EC018A819B81892B19F480E090E005
:1019600018C0ED01EE81FF814191FF83EE838A81F2
:101970009B8101979B838A83288539858D919C91D2
:10198000820F931FE817F90710F03F832E83842FEF
:101990009927DF91CF910895FC01518340831382F1
:1019A0001282758364837783668371876087089565
:1019B000FC0182819381892B19F480E090E00895E5
:1019C0000680F781E02D808199270895CF93DF93DA
:1019D000DC01EC012A813B818D919C9111972817A4
:1019E0003907A8F4EC81FD816193FD83EC838A8142
:1019F0009B8101969B838A83288539858D919C9153
:101A0000820F931FE817F90710F03D832C83DF91B5
:101A1000CF910895CF93DF93DC01EC018A819B8104
:101A2000892B19F440E050E019C0ED01EE81FF81EF
:101A300041915191FF83EE838A819B8101979B8322
:101A40008A83288539858D919C91880F991F820FF3
:101A5000931FE817F90710F03F832E83CA01DF9127
:101A6000CF910895FC0151834083138212827583C4
:101A7000648377836683718760870895FC01828120
:101A80009381892B19F480E090E008950680F78116
:101A9000E02D808191810895CF93DF93DC01EC01EB
:101AA0002A813B818D919C91119728173907C0F4A9
:101AB000EC81FD8161937193FD83EC838A819B812D
:101AC00001969B838A83288539858D919C91880F07
:101AD000991F820F931FE817F90710F03D832C839D
:101AE000DF91CF9108953F924F925F926F927F92D4
:101AF0008F929F92AF92BF92CF92DF92EF92FF921E
:101B00000F931F93CF93DF938C012B01EA01611593
:101B1000710519F0FB0191838083209749F0CE0174
:101B20000297839728F060E070E080E090E0F6C0D4
:101B3000F801E1908F018E2D99270E946514892B61
:101B4000B9F7FDE2EF1631F4F801E1908F0181E081
:101B5000382E07C0FBE2EF1619F4F801E1908F016F
:101B60003324209719F0C031D105C1F4F0E3EF160A
:101B700079F4F8018081883711F0883549F4F8014B
:101B8000E1800E5F1F4FF2E03F2AC0E1D0E006C0C7
:101B9000209721F480E3E816E9F427C0C830D10586
:101BA00031F1C930D10524F4C230D10531F50CC072
:101BB000CA30D10589F0C031D105F9F4A12CB12C7E
:101BC000C12CB8E0DB2E26C0A12CB12CC12CA0E486
:101BD000DA2E20C0CAE0D0E0FCECAF2EFCECBF2E29
:101BE000FCECCF2EFCE0DF2E15C0C8E0D0E0A12C2D
:101BF000B12CC12CE0E1DE2E0DC09E01442737FD43
:101C00004095542F60E070E080E090E80E9443141B
:101C100059016A0120E030E040E050E060E03E0120
:101C2000882477FC8094982C70EDF72EFE0CE9E068
:101C3000EF1570F48E2D81548A3118F499ECF92E39
:101C400006C08E2D81568A3150F589EAF82EFE0C99
:101C50008F2D99278C179D0714F567FD1CC0A216C0
:101C6000B306C406D506B0F0CA01B901A4019301B8
:101C70000E9477149B01AC012F0D311D411D511D98
:101C80002130F0E03F07F0E04F07F0E85F0710F485
:101C900061E001C06FEFF801E1908F01C5CF411401
:101CA000510481F0662331F001501040F20111839C
:101CB000008308C031FE1AC002501040F2011183A7
:101CC000008314C067FF12C030FE05C020E030E082
:101CD00040E050E804C02FEF3FEF4FEF5FE782E2B4
:101CE00090E090932A038093290316C030FE08C029
:101CF00050954095309521953F4F4F4F5F4F0CC009
:101D000057FF0AC082E290E090932A038093290350
:101D10002FEF3FEF4FEF5FE7CA01B901DF91CF919E
:101D20001F910F91FF90EF90DF90CF90BF90AF90F9
:101D30009F908F907F906F905F904F903F9008950D
:101D4000FB01DC018D910590602D502D50625136C4
:101D500024F05B3714F460628062861B11F400206B
:101D600089F7990B0895FB01DC018D910190801991
:101D700011F40020D1F7990B0895FB01DC010190CB
:101D80000D920020E1F70895EF92FF920F931F93B9
:101D9000CF93DF938C017B01892B11F4672BD1F159
:101DA0006EE070E081E090E00E949912FC010097E3
:101DB00089F1DC0180E88383E114F10471F0F3869A
:101DC000E28681E883838091230390912403892B09
:101DD00021F4F0932403E093230301151105E1F0AE
:101DE000118700878381826083838091250390918E
:101DF0002603892B89F4F0932603E0932503809131
:101E0000270390912803892B39F4F0932803E0935A
:101E1000270302C0A0E0B0E0CD01DF91CF911F9178
:101E20000F91FF90EF900895CF93DF93CDB7DEB77A
:101E300022970FB6F894DEBF0FBECDBFFE013796D6
:101E400061917191FA83E983AF01809125039091AB
:101E500026030E94CE0F22960FB6F894DEBF0FBE67
:101E6000CDBFDF91CF910895CF93DF93CDB7DEB78C
:101E700022970FB6F894DEBF0FBECDBFFE01379696
:101E800061917191FA83E983E0912503F091260332
:101E900083818860838349815A8180912503909151
:101EA00026030E94CE0FE0912503F09126032381A3
:101EB000277F238322960FB6F894DEBF0FBECDBFD7
:101EC000DF91CF91089560912503709126030E94C0
:101ED000D41308950F931F93CF93DF93CDB7DEB73D
:101EE00060970FB6F894DEBF0FBECDBF0F89188D77
:101EF00086E08E831C830B838FEF9FE798878F8309
:101F0000AE01455E5F4F5A834983698D7A8DCE015C
:101F100003960E94CE0F29853A85020F131FF80100
:101F2000108260960FB6F894DEBF0FBECDBFDF9172
:101F3000CF911F910F9108950F931F93CF93DF932C
:101F4000CDB7DEB760970FB6F894DEBF0FBECDBF3A
:101F50000F89188D8EE08E831C830B838FEF9FE794
:101F600098878F83AE01455E5F4F5A834983698DA1
:101F70007A8DCE0103960E94CE0F29853A85020FF5
:101F8000131FF801108260960FB6F894DEBF0FBEE3
:101F9000CDBFDF91CF911F910F9108952F923F9266
:101FA0004F925F926F927F928F929F92AF92BF9269
:101FB000CF92DF92EF92FF920F931F93CF93DF9315
:101FC000CDB7DEB764970FB6F894DEBF0FBECDBFB6
:101FD000CC24DD2476011C017C8B6B8B2A01FC0157
:101FE00017821682838181FD03C08FEF9FEF88C225
:101FF000AA24BB2472C2A0FE57C28A8980538A30A9
:10200000E8F4FA89F03341F42D85222329F4A3FC66
:1020100003C080E091E06FC08AE0ED85E802C00176
:102020001124FA89F80FF053FD87F7FF02C02FE75C
:102030002D87A3FC4CC23D853E8749C2C5018870EF
:102040009070A3FE05C0ED85EE2311F4F1E0FD874D
:102050002A89283624F525360CF05BC0233509F48F
:1020600080C024358CF42B32C1F12C3234F4203270
:10207000C1F1233209F00DC23CC03A893D32B1F1C1
:102080003E3209F006C23AC08A89833609F449C053
:1020900084360CF081C0883509F0FBC11BC0EA8989
:1020A000E03709F4A3C0E13744F4EC3669F1EF36C8
:1020B00071F0E93609F0EDC16FC0FA89F53709F41E
:1020C0009DC0F83739F0F33709F0E3C134C028E098
:1020D000298B94C030E1398B91C080E190E0A82A2F
:1020E000B92AE0E2F0E0AE2ABF2AF1C120E830E0F0
:1020F0000DC080E490E0A82AB92AE9C1E8E0F0E048
:10210000AE2ABF2A1D86E3C124E030E0A22AB32A0A
:10211000DEC14FE3C42E3E8531503E8783E68A8B75
:1021200044C1F201C080FE85F150FE8722E030E01C
:10213000420E531E3AC1F201C080D180892B49F072
:10214000FD856F2F772767FD7095C6010E94C91323
:1021500019C0F60101900020E9F73197EC19E98BDD
:1021600012C0F201C080D180892B49F0FD856F2F0C
:10217000772767FD7095C6010E94B71303C0C6019B
:102180000E94AE13898B22E030E0420E531E3E8542
:102190008989381B3E8709C1A2FE08C0F2018081EF
:1021A0009181A281B38124E030E009C0F2018081F5
:1021B0009181AA2797FDA095BA2F22E030E0420E28
:1021C000531E6C017D01B7FF0CC082E090E0A82A8D
:1021D000B92AF094E094D094C094C11CD11CE11CA5
:1021E000F11CEFEBFFEFAE22BF2221C020E430E074
:1021F000A22AB32A38E73A8B80E1898BA2FE08C075
:10220000F20180819181A281B38124E030E007C096
:10221000F20180819181AA27BB2722E030E0420EA3
:10222000531E6C017D018FEC9FEFA822B92287011C
:102230007601FE013196F88BEF87F9896F2E7724AE
:1022400088249924C801B701A40193010E94431472
:102250006A3024F02A89620F615201C0605DEF8507
:10226000F8896193F88BEF87C801B701A401930146
:102270000E94431479018A01211531054105510558
:1022800009F7CC24DD247601CE010196CF84C81A4B
:10229000C50182739070892B19F0FE85F150FE877D
:1022A000A6FE09C02989203111F482E001C081E035
:1022B0003E85381B3E8738E0832E912C8A209B2058
:1022C000A3FE1BC08D85282F332727FD30958C2D2D
:1022D00099278217930754F0E7EFFFEFAE22BF2252
:1022E00028E0822E912C8A209B2007C0FD85FC19B6
:1022F000FD872E852F1B2E8703C03E853C193E8708
:10230000C50180789170892B69F48E8506C0B10172
:1023100080E290E00E94D413812F182F11501816DC
:10232000B4F31E87A1FE04C0B1018DE290E00BC0A2
:10233000A4FE04C0B1018BE290E005C0A5FE05C07B
:10234000B10180E290E00E94D413A6FE10C0B1015A
:1023500080E390E00E94D4138989803141F4B10177
:10236000EA898E2F992787FD90950E94D413B0FE9D
:102370000DC08E8506C0B10180E390E00E94D413A9
:10238000812F182F11501816B4F31E87892869F071
:102390002D8506C0B10180E390E00E94D413212F67
:1023A000122F11501216B4F31D8790E8692E712C6C
:1023B0006A207B20A7FC0DC08E8506C0B10180E29B
:1023C00090E00E94D413812F182F11501816B4F3E7
:1023D0001E87FA89F33641F4B1018C2D992787FDC8
:1023E00090950E94D41345C02A892337B1F4460141
:1023F0005601198909C0F50181915F01B101992741
:1024000087FD90950E94D4131150A8F76401F989B3
:10241000CF0ED11C2FEF298B2CC03A89333519F000
:102420000F8518891FC046018601B98808C0F801C8
:102430008491B10199270E94D4130F5F1F4FBA9462
:10244000FFEFBF16A1F764012989C20ED11CF98BD9
:1024500010C0F80182918F01B101992787FD9095F5
:102460000E94D413CE0101960817190791F7188B13
:102470000F876728B1F08E8506C0B10180E290E039
:102480000E94D413812F182F11501816B4F31E87F1
:1024900008C0B101FA898F2F992787FD90950E9476
:1024A000D413AA24BB2413C02A89253241F43AE06C
:1024B000398B1E861D8681E0A82EB12C08C0B10183
:1024C000EA898E2F992787FD90950E94D4132B8936
:1024D0003C892F5F3F4F3C8B2B8BF101838183FF26
:1024E00004C0EB89FC89F49103C0EB89FC89F0817D
:1024F000FA8B2A89222309F07ECDF101868197810A
:1025000064960FB6F894DEBF0FBECDBFDF91CF91BA
:102510001F910F91FF90EF90DF90CF90BF90AF9001
:102520009F908F907F906F905F904F903F902F90F3
:1025300008950F931F93CF93DF93869F8001879F0A
:10254000100D969F100D1124C8010E94B512EC01C8
:10255000009729F0A80160E070E00E94C213CE014C
:10256000DF91CF911F910F910895CF93DF93AC012D
:10257000029710F442E050E0A0912D03B0912E0399
:10258000FD01C0E0D0E020E030E020C080819181FA
:102590008417950769F482819381209719F09B83B2
:1025A0008A8304C090932E0380932D03CF0132C001
:1025B0004817590738F42115310519F08217930788
:1025C00008F49C01EF010280F381E02D3097F1F6D1
:1025D0002115310589F1C901841B950B049708F475
:1025E000A901E0E0F0E026C08D919C91119782173F
:1025F0009307E9F44817590779F4ED018A819B8123
:10260000309719F09383828304C090932E038093B4
:102610002D03CD01029649C0841B950BFD01E80FE7
:10262000F91F4193519302978D939C933AC0FD01FA
:10263000A281B3811097C1F680912B0390912C0356
:10264000892B41F4809170019091710190932C033A
:1026500080932B0320917201309173012115310574
:1026600041F42DB73EB780916E0190916F01281B08
:10267000390BE0912B03F0912C032E1B3F0B2417F9
:10268000350788F0CA0102962817390760F0CF0194
:10269000840F951F029690932C0380932B034193F4
:1026A0005193CF0102C080E090E0DF91CF91089577
:1026B000CF93DF93009709F44EC0EC0122971B8261
:1026C0001A82A0912D03B0912E03109711F140E0D2
:1026D00050E001C0DC01AC17BD0700F1BB83AA8349
:1026E000FE0121913191E20FF31FEA17FB0771F40C
:1026F0002E5F3F4F8D919C911197820F931F99836D
:102700008883FD01828193819B838A8341155105D2
:1027100059F4D0932E03C0932D031DC0FD01828177
:102720009381AD010097B1F6FA01D383C283219161
:102730003191E20FF31FEC17FD0769F42E5F3F4F55
:1027400088819981820F931FFA01918380838A8106
:102750009B8193838283DF91CF910895FC01059043
:102760000020E9F7809590958E0F9F1F0895FC013A
:102770000590615070400110D8F7809590958E0FAC
:102780009F1F0895DC0101C06D9341505040E0F758
:102790000895FC016150704001900110D8F78095B8
:1027A00090958E0F9F1F08950F931F93CF93DF93E4
:1027B0008C01EB018B81992781FF1BC082FF0DC02B
:1027C0002E813F818C819D812817390764F4E8812F
:1027D000F9810193F983E88306C0E885F985802FA4
:1027E0000995892B31F48E819F8101969F838E8379
:1027F00002C00FEF1FEFC801DF91CF911F910F9122
:102800000895AA1BBB1B51E107C0AA1FBB1FA61737
:10281000B70710F0A61BB70B881F991F5A95A9F789
:1028200080959095BC01CD01089597FB092E072650
:102830000AD077FD04D0E5DF06D000201AF47095A9
:1028400061957F4F0895F6F7909581959F4F089574
:1028500097FB092E05260ED057FD04D014D00AD0C0
:10286000001C38F450954095309521953F4F4F4FBF
:102870005F4F0895F6F790958095709561957F4F1D
:102880008F4F9F4F0895A1E21A2EAA1BBB1BFD017B
:102890000DC0AA1FBB1FEE1FFF1FA217B307E4073F
:1028A000F50720F0A21BB30BE40BF50B661F771F97
:1028B000881F991F1A9469F7609570958095909577
:1028C0009B01AC01BD01CF01089591110DC0803273
:1028D00051F08A3041F08C3031F08D3021F0893068
:1028E00011F08B3099F70895992788270895629FF2
:1028F000D001739FF001829FE00DF11D649FE00DF8
:10290000F11D929FF00D839FF00D749FF00D659F58
:10291000F00D9927729FB00DE11DF91F639FB00D57
:0C292000E11DF91FBD01CF011124089535
:10292C002533753A252D3673203A20252D323273F6
:10293C00002533753A252D3673003F00616E6E6F9E
:10294C00756E636500737065616B696E6720002539
:10295C007520006C697374006C6973747600736312
:10296C0070007769640063616E277420726561641E
:10297C0020776964746820272573270A00776964B7
:10298C00203D2025750A002573200050960220005A
:04299C002F03000005
:00000001FF
